:020000020000FC
:0200000006C137
:020008005DC0D9
:10000E0018C001020507446F75626C65466F782053
:10001E004D756C7469706C657865724120526576A9
:10002E002E20312E30610D0000006572726F720D40
:10003E0000006FB6ACB15C9909C082FD13C081FFA0
:10004E0007C0AD3009F48D7F8A2E88606FBE18957B
:10005E008260A43221F08A2E88606FBE189584606B
:10006E006FBE18958B7FA43221F48A2E88606FBEE6
:10007E0018958D7FA03379F0A13389F0A23399F0D2
:10008E00A333A9F0AF3321F0A33711F06FBE18954B
:10009E00EA2E6FBE1895A2E07A2E6FBE1895A4E0D8
:1000AE007A2E6FBE1895A0E27A2E6FBE1895A0E834
:1000BE007A2E6FBE18956FB680FD03C083FD15C0F6
:1000CE0020C06A95F1F4DD2011F48E7F1AC0DA9407
:1000DE005694A8B320F0A729A8BB68E012C070946C
:1000EE00A7217094A8BB68E00CC0877F8160582C54
:1000FE00509469E0D62E68E0A8B37094A72170944E
:10010E00A8BBA6B374FD13C0A0FF0CC01AC0BA2FB3
:10011E00B17019F47F7E906114C07F7E8061109261
:10012E00C4000FC07061B9E09B2E2AE00AC02150B6
:10013E0041F49A9461F3BA2FB170B095BF5F1794E2
:10014E0028E075FD13C0A3FF0CC01AC0BA2FB870FB
:10015E0019F47F7D906214C07F7D80622092C5006D
:10016E000FC07062B9E0AB2E3AE00AC0315041F4D4
:10017E00AA9461F3BA2FB870B095BF5F279438E098
:10018E0076FD13C0A4FF0CC01AC0BA2FB07119F4BB
:10019E007F7B906414C07F7B80643092C6000FC05A
:1001AE007064B9E0BB2E4AE00AC0415041F4BA94E3
:1001BE0061F3BA2FB071B095BF5F379448E077FD09
:1001CE0013C0A6FF0CC01AC0BA2FB07419F47F77F3
:1001DE00906814C07F7780684092C7000FC0706827
:1001EE00B9E0CB2E5AE00AC0515041F4CA9461F3E3
:1001FE00BA2FB074B095BF5F479458E06FBE189594
:10020E000FED0DBF06EA07BB0FEF08BB08E90AB9F1
:10021E0000E409B900270FBD09E00EBD00270BBD94
:10022E0001E80ABD00E409BF02E0702E00E600936B
:10023E00C80009E70093C90002E90093CA000BEA5F
:10024E000093CB00EE248827772766249927DD2498
:10025E00DA94FF27DD27789490D070FF13C05D9954
:10026E0002C08BD0FCCF00E30CB9E0E65D9902C072
:10027E0084D0FCCF01910CB90D30C1F77E7F00E622
:10028E000093C8007AD071FF13C05D9902C075D07B
:10029E00FCCF01E30CB9E9E75D9902C06ED0FCCF4B
:1002AE0001910CB90D30C1F77D7F09E70093C900AC
:1002BE0064D072FF13C05D9902C05FD0FCCF02E321
:1002CE000CB9E2E95D9902C058D0FCCF01910CB98E
:1002DE000D30C1F77B7F02E90093CA004ED073FF49
:1002EE0013C05D9902C049D0FCCF03E30CB9EBEA11
:1002FE005D9902C042D0FCCF01910CB90D30C1F70F
:10030E00777F0BEA0093CB00EE2009F4A5CF0E2DDC
:10031E000F3379F00337D1F0E8E35D9902C02DD0A9
:10032E00FCCFC895E395002D0CB90D30B1F7EE2436
:10033E0093CFE4E15D9902C020D0FCCFC895E39540
:10034E00002D0CB90D30B1F7EE2486CFD8E0C92FB1
:10035E005D9902C012D0FCCFCC0F10F401E301C0A6
:10036E0000E30CB9DA95A1F7EE2499275D9902C046
:10037E0004D0FCCF0DE00CB96FCF84FF12C070FF1C
:10038E0002C090610EC00091C400C091C8000993D4
:10039E00C93708F0C0E6C093C8008F7E0D3009F44F
:1003AE00716085FF12C071FF02C090620EC0009195
:1003BE00C500C091C9000993C23908F0C9E7C093BE
:1003CE00C9008F7D0D3009F4726086FF12C072FF76
:1003DE0002C090640EC00091C600C091CA0009937D
:1003EE00CB3A08F0C2E9C093CA008F7B0D3009F4F6
:1003FE00746087FF12C073FF02C090680EC0009138
:10040E00C700C091CB000993C43C08F0CBEAC0935F
:0C041E00CB008F770D3009F47860089552
:00000001FF
